BL51 BANKED LINKER/LOCATER V6.22.2.0                                                    10/25/2022  13:54:05  PAGE 1


BL51 BANKED LINKER/LOCATER V6.22.2.0, INVOKED BY:
C:\KEIL_V5\C51\BIN\BL51.EXE .\Release\system_FE81001.obj, .\Release\STARTUP.obj, .\Release\main.obj TO .\Release\Sample_
>> DrvSDM_MultiB REGFILE (.\Release\Sample_DrvSDM_MultiB.ORC) PRINT (.\Sample_DrvSDM_MultiB.m51) RAMSIZE (256) CODE (0X0
>> 000-0X1FFF) XDATA (0X8000-0X87FF)


MEMORY MODEL: SMALL WITH FLOATING POINT ARITHMETIC


INPUT MODULES INCLUDED:
  .\Release\system_FE81001.obj (SYSTEM_FE81001)
  .\Release\STARTUP.obj (?C_STARTUP)
  .\Release\main.obj (MAIN)
  C:\KEIL_V5\C51\LIB\C51FPS.LIB (?C?FPADD)
  C:\KEIL_V5\C51\LIB\C51FPS.LIB (?C?FPMUL)
  C:\KEIL_V5\C51\LIB\C51FPS.LIB (?C?FPDIV)
  C:\KEIL_V5\C51\LIB\C51FPS.LIB (?C?FCAST)
  C:\KEIL_V5\C51\LIB\C51FPS.LIB (?C?CASTF)
  C:\KEIL_V5\C51\LIB\C51FPS.LIB (?C?FPGETOPN)
  C:\KEIL_V5\C51\LIB\C51S.LIB (?C_INIT)
  C:\KEIL_V5\C51\LIB\C51S.LIB (?C?UIDIV)
  C:\KEIL_V5\C51\LIB\C51S.LIB (?C?LMUL)
  C:\KEIL_V5\C51\LIB\C51S.LIB (?C?LNEG)
  C:\KEIL_V5\C51\LIB\C51S.LIB (?C?ULCMP)
  C:\KEIL_V5\C51\LIB\C51S.LIB (?C?ICASE)
  C:\KEIL_V5\C51\LIB\C51S.LIB (?C_IBP)


LINK MAP OF MODULE:  .\Release\Sample_DrvSDM_MultiB (SYSTEM_FE81001)


            TYPE    BASE      LENGTH    RELOCATION   SEGMENT NAME
            -----------------------------------------------------

            * * * * * * *   D A T A   M E M O R Y   * * * * * * *
            REG     0000H     0008H     ABSOLUTE     "REG BANK 0"
            DATA    0008H     0040H     UNIT         ?DT?MAIN
            DATA    0048H     0006H     UNIT         ?DT?_DELAY?MAIN
            DATA    004EH     0002H     UNIT         ?DT?_DIG1?MAIN
            DATA    0050H     0002H     UNIT         ?DT?_DIG2?MAIN
            DATA    0052H     0002H     UNIT         ?DT?_DIG3?MAIN
            DATA    0054H     0002H     UNIT         ?DT?_DIG4?MAIN
            DATA    0056H     0002H     UNIT         ?DT?MAIN?MAIN
            DATA    0058H     0001H     UNIT         ?DT?SDMISR?MAIN
            DATA    0059H     0001H     UNIT         ?DT?LCMINIT?MAIN
            DATA    005AH     0001H     UNIT         ?C?LIB_DATA
            IDATA   005BH     0001H     UNIT         ?STACK

            * * * * * * *  X D A T A   M E M O R Y  * * * * * * *
                    0000H     8000H                  *** GAP ***
            XDATA   8000H     0004H     UNIT         ?XD?MAIN

            * * * * * * *   C O D E   M E M O R Y   * * * * * * *
            CODE    0000H     0003H     ABSOLUTE     
            CODE    0003H     0028H     UNIT         ?PR?SDM_LIGHT_CONFIG?MAIN
            CODE    002BH     0003H     ABSOLUTE     
            CODE    002EH     044DH     UNIT         ?C?LIB_CODE
            CODE    047BH     021CH     UNIT         ?PR?IOCONFIG?MAIN
BL51 BANKED LINKER/LOCATER V6.22.2.0                                                  10/25/2022  13:54:05  PAGE 2


            CODE    0697H     01BBH     UNIT         ?PR?MAIN?MAIN
            CODE    0852H     0128H     UNIT         ?PR?RTD_MEASURE_SHOW?MAIN
            CODE    097AH     00D6H     UNIT         ?PR?RTD_SHOW?MAIN
            CODE    0A50H     00B8H     UNIT         ?PR?_DIG1?MAIN
            CODE    0B08H     00B8H     UNIT         ?PR?_DIG2?MAIN
            CODE    0BC0H     00B8H     UNIT         ?PR?_DIG3?MAIN
            CODE    0C78H     00B8H     UNIT         ?PR?_DIG4?MAIN
            CODE    0D30H     00B3H     UNIT         ?PR?SDMISR?MAIN
            CODE    0DE3H     009DH     UNIT         ?C_C51STARTUP
            CODE    0E80H     008BH     UNIT         ?PR?SDMCONFIG?MAIN
            CODE    0F0BH     0085H     UNIT         ?PR?CLKCONFIG?MAIN
            CODE    0F90H     0065H     UNIT         ?C_INITSEG
            CODE    0FF5H     004EH     UNIT         ?PR?ANACCONFIG?MAIN
            CODE    1043H     0046H     UNIT         ?PR?TMR0INIT?MAIN
            CODE    1089H     0046H     UNIT         ?PR?TMR1INIT?MAIN
            CODE    10CFH     003CH     UNIT         ?PR?LCMINIT?MAIN
            CODE    110BH     003BH     UNIT         ?PR?_DELAY?MAIN
            CODE    1146H     0026H     UNIT         ?PR?LIGHT_SHOW?MAIN
            CODE    116CH     000CH     UNIT         ?PR?POINT?MAIN
            CODE    1178H     0004H     UNIT         ?PR?TIMERINIT?MAIN
            CODE    117CH     0001H     UNIT         ?PR?SYSTEMINIT?SYSTEM_FE81001



OVERLAY MAP OF MODULE:   .\Release\Sample_DrvSDM_MultiB (SYSTEM_FE81001)


SEGMENT
  +--> CALLED SEGMENT
---------------------
?C_C51STARTUP
  +--> ?PR?MAIN?MAIN
  +--> ?C_INITSEG

?PR?MAIN?MAIN
  +--> ?PR?CLKCONFIG?MAIN
  +--> ?PR?IOCONFIG?MAIN
  +--> ?PR?LCMINIT?MAIN
  +--> ?PR?ANACCONFIG?MAIN
  +--> ?PR?SDMCONFIG?MAIN
  +--> ?PR?TIMERINIT?MAIN
  +--> ?PR?_DELAY?MAIN
  +--> ?PR?RTD_MEASURE_SHOW?MAIN
  +--> ?PR?RTD_SHOW?MAIN
  +--> ?PR?SDM_LIGHT_CONFIG?MAIN
  +--> ?PR?LIGHT_SHOW?MAIN

?PR?TIMERINIT?MAIN
  +--> ?PR?TMR0INIT?MAIN

?PR?RTD_SHOW?MAIN
  +--> ?PR?_DIG1?MAIN
  +--> ?PR?_DIG2?MAIN
  +--> ?PR?POINT?MAIN
  +--> ?PR?_DIG3?MAIN
  +--> ?PR?_DIG4?MAIN

BL51 BANKED LINKER/LOCATER V6.22.2.0                                                  10/25/2022  13:54:05  PAGE 3




SYMBOL TABLE OF MODULE:  .\Release\Sample_DrvSDM_MultiB (SYSTEM_FE81001)

  VALUE           TYPE          NAME
  ----------------------------------

  -------         MODULE        SYSTEM_FE81001
  C:0000H         SYMBOL        _ICE_DUMMY_
  C:117CH         PUBLIC        SystemInit
  -------         PROC          SYSTEMINIT
  C:117CH         LINE#         38
  C:117CH         LINE#         39
  C:117CH         LINE#         41
  -------         ENDPROC       SYSTEMINIT
  -------         ENDMOD        SYSTEM_FE81001

  -------         MODULE        ?C_STARTUP
  C:0DE3H         SEGMENT       ?C_C51STARTUP
  I:005BH         SEGMENT       ?STACK
  C:0000H         PUBLIC        ?C_STARTUP
  D:00E0H         SYMBOL        ACC
  D:00F0H         SYMBOL        B
  D:0083H         SYMBOL        DPH
  D:0082H         SYMBOL        DPL
  N:0001H         SYMBOL        IBPSTACK
  N:0100H         SYMBOL        IBPSTACKTOP
  N:0080H         SYMBOL        IDATALEN
  C:0DE6H         SYMBOL        IDATALOOP
  N:0000H         SYMBOL        PBPSTACK
  N:0100H         SYMBOL        PBPSTACKTOP
  N:0000H         SYMBOL        PDATALEN
  N:0000H         SYMBOL        PDATASTART
  N:0000H         SYMBOL        PPAGE
  N:0000H         SYMBOL        PPAGEENABLE
  D:00A0H         SYMBOL        PPAGE_SFR
  D:0081H         SYMBOL        SP
  C:0DE3H         SYMBOL        STARTUP1
  N:0000H         SYMBOL        XBPSTACK
  N:0000H         SYMBOL        XBPSTACKTOP
  N:0800H         SYMBOL        XDATALEN
  C:0DF1H         SYMBOL        XDATALOOP
  N:8000H         SYMBOL        XDATASTART
  C:0000H         LINE#         126
  C:0DE3H         LINE#         133
  C:0DE5H         LINE#         134
  C:0DE6H         LINE#         135
  C:0DE7H         LINE#         136
  C:0DE9H         LINE#         140
  C:0DECH         LINE#         141
  C:0DEEH         LINE#         145
  C:0DF0H         LINE#         147
  C:0DF1H         LINE#         148
  C:0DF2H         LINE#         149
  C:0DF3H         LINE#         150
  C:0DF5H         LINE#         151
  C:0DF7H         LINE#         170
BL51 BANKED LINKER/LOCATER V6.22.2.0                                                  10/25/2022  13:54:05  PAGE 4


  C:0DFAH         LINE#         185
  C:0DFDH         LINE#         196
  -------         ENDMOD        ?C_STARTUP

  -------         MODULE        MAIN
  C:0000H         SYMBOL        _ICE_DUMMY_
  D:0090H         PUBLIC        P1
  D:00B0H         PUBLIC        P3
  D:0008H         PUBLIC        alpha
  D:00A8H         PUBLIC        IE
  C:097AH         PUBLIC        RTD_show
  C:110BH         PUBLIC        _delay
  D:000CH         PUBLIC        Temp
  D:000EH         PUBLIC        flag_light
  D:00B8H         PUBLIC        IP
  C:1178H         PUBLIC        TimerInit
  C:0697H         PUBLIC        main
  D:000FH         PUBLIC        Temp_0
  D:0011H         PUBLIC        Temp_1
  X:8000H         PUBLIC        R0_ADC
  D:0013H         PUBLIC        count
  C:116CH         PUBLIC        point
  D:0098H         PUBLIC        SCON
  C:0F0BH         PUBLIC        CLKConfig
  D:0088H         PUBLIC        TCON
  D:0015H         PUBLIC        Temp_avg
  C:0003H         PUBLIC        SDM_light_config
  C:1043H         PUBLIC        TMR0Init
  C:1089H         PUBLIC        TMR1Init
  C:1146H         PUBLIC        light_show
  C:0E80H         PUBLIC        SDMConfig
  D:0017H         PUBLIC        bb
  D:0019H         PUBLIC        flag_ADC
  C:0A50H         PUBLIC        _Dig1
  C:0B08H         PUBLIC        _Dig2
  C:0BC0H         PUBLIC        _Dig3
  D:001AH         SYMBOL        raw_data
  C:0C78H         PUBLIC        _Dig4
  C:0D30H         PUBLIC        SDMISR
  D:001DH         PUBLIC        b
  C:0852H         PUBLIC        RTD_measure_show
  D:0021H         PUBLIC        flag_RTD
  D:00C8H         PUBLIC        T2CON
  C:0FF5H         PUBLIC        ANACConfig
  C:047BH         PUBLIC        IOConfig
  C:10CFH         PUBLIC        LCMInit
  D:0022H         PUBLIC        PWM_UP
  D:0044H         PUBLIC        R_ADC
  D:00D0H         PUBLIC        PSW
  -------         PROC          _DELAY
  D:0048H         SYMBOL        cnt
  -------         DO            
  D:004AH         SYMBOL        i
  D:004CH         SYMBOL        j
  -------         ENDDO         
  C:110BH         LINE#         63
  C:110FH         LINE#         64
BL51 BANKED LINKER/LOCATER V6.22.2.0                                                  10/25/2022  13:54:05  PAGE 5


  C:110FH         LINE#         67
  C:1120H         LINE#         68
  C:1145H         LINE#         70
  -------         ENDPROC       _DELAY
  -------         PROC          SDMISR
  -------         DO            
  D:0058H         SYMBOL        int_stat
  -------         ENDDO         
  C:0D30H         LINE#         82
  C:0D4DH         LINE#         84
  C:0D54H         LINE#         86
  C:0D5AH         LINE#         89
  C:0D61H         LINE#         90
  C:0D68H         LINE#         91
  C:0D6FH         LINE#         93
  C:0DC5H         LINE#         95
  C:0DC8H         LINE#         99
  -------         ENDPROC       SDMISR
  -------         PROC          LCMINIT
  -------         DO            
  D:0059H         SYMBOL        i
  -------         ENDDO         
  C:10CFH         LINE#         102
  C:10CFH         LINE#         103
  C:10CFH         LINE#         107
  C:10DAH         LINE#         110
  C:10E0H         LINE#         113
  C:10F2H         LINE#         114
  C:1100H         LINE#         115
  C:1104H         LINE#         117
  C:110AH         LINE#         119
  -------         ENDPROC       LCMINIT
  -------         PROC          SDMCONFIG
  C:0E80H         LINE#         130
  C:0E80H         LINE#         131
  C:0E80H         LINE#         135
  C:0E85H         LINE#         138
  C:0E96H         LINE#         141
  C:0EA7H         LINE#         144
  C:0EB2H         LINE#         147
  C:0EBDH         LINE#         150
  C:0ED3H         LINE#         153
  C:0EF4H         LINE#         156
  C:0EFFH         LINE#         159
  C:0F0AH         LINE#         161
  -------         ENDPROC       SDMCONFIG
  -------         PROC          SDM_LIGHT_CONFIG
  C:0003H         LINE#         163
  C:0003H         LINE#         164
  C:0003H         LINE#         165
  C:0014H         LINE#         167
  C:002AH         LINE#         168
  -------         ENDPROC       SDM_LIGHT_CONFIG
  -------         PROC          LIGHT_SHOW
  C:1146H         LINE#         170
  C:1146H         LINE#         171
  C:1146H         LINE#         172
BL51 BANKED LINKER/LOCATER V6.22.2.0                                                  10/25/2022  13:54:05  PAGE 6


  C:1149H         LINE#         174
  C:115FH         LINE#         175
  C:115FH         LINE#         176
  C:1164H         LINE#         177
  C:1165H         LINE#         180
  C:1165H         LINE#         181
  C:116BH         LINE#         182
  C:116BH         LINE#         184
  -------         ENDPROC       LIGHT_SHOW
  -------         PROC          ANACCONFIG
  C:0FF5H         LINE#         197
  C:0FF5H         LINE#         198
  C:0FF5H         LINE#         200
  C:1000H         LINE#         201
  C:100BH         LINE#         202
  C:1016H         LINE#         205
  C:1021H         LINE#         208
  C:102CH         LINE#         211
  C:1037H         LINE#         214
  C:1042H         LINE#         216
  -------         ENDPROC       ANACCONFIG
  -------         PROC          IOCONFIG
  C:047BH         LINE#         227
  C:047BH         LINE#         228
  C:047BH         LINE#         230
  C:049CH         LINE#         233
  C:04BDH         LINE#         238
  C:04DEH         LINE#         241
  C:04FFH         LINE#         244
  C:0520H         LINE#         247
  C:0536H         LINE#         250
  C:054CH         LINE#         253
  C:0562H         LINE#         256
  C:0578H         LINE#         259
  C:058EH         LINE#         262
  C:05A4H         LINE#         265
  C:05BAH         LINE#         268
  C:05D0H         LINE#         271
  C:05E6H         LINE#         274
  C:05FCH         LINE#         277
  C:0612H         LINE#         280
  C:0628H         LINE#         283
  C:0649H         LINE#         286
  C:065FH         LINE#         287
  C:0675H         LINE#         289
  C:0696H         LINE#         292
  -------         ENDPROC       IOCONFIG
  -------         PROC          CLKCONFIG
  C:0F0BH         LINE#         304
  C:0F0BH         LINE#         305
  C:0F0BH         LINE#         307
  C:0F16H         LINE#         310
  C:0F21H         LINE#         311
  C:0F2CH         LINE#         314
  C:0F42H         LINE#         317
  C:0F4DH         LINE#         320
  C:0F63H         LINE#         321
BL51 BANKED LINKER/LOCATER V6.22.2.0                                                  10/25/2022  13:54:05  PAGE 7


  C:0F79H         LINE#         324
  C:0F84H         LINE#         325
  C:0F8FH         LINE#         327
  -------         ENDPROC       CLKCONFIG
  -------         PROC          _DIG1
  D:004EH         SYMBOL        num
  C:0A50H         LINE#         329
  C:0A54H         LINE#         330
  C:0A54H         LINE#         331
  C:0A88H         LINE#         332
  C:0A88H         LINE#         334
  C:0A88H         LINE#         335
  C:0A8EH         LINE#         336
  C:0A94H         LINE#         337
  C:0A95H         LINE#         339
  C:0A95H         LINE#         340
  C:0A9AH         LINE#         341
  C:0AA0H         LINE#         342
  C:0AA1H         LINE#         344
  C:0AA1H         LINE#         345
  C:0AA7H         LINE#         346
  C:0AADH         LINE#         347
  C:0AAEH         LINE#         349
  C:0AAEH         LINE#         350
  C:0AB4H         LINE#         351
  C:0ABAH         LINE#         352
  C:0ABBH         LINE#         354
  C:0ABBH         LINE#         355
  C:0AC1H         LINE#         356
  C:0AC7H         LINE#         357
  C:0AC8H         LINE#         359
  C:0AC8H         LINE#         360
  C:0ACEH         LINE#         361
  C:0AD4H         LINE#         362
  C:0AD5H         LINE#         364
  C:0AD5H         LINE#         365
  C:0ADBH         LINE#         366
  C:0AE1H         LINE#         367
  C:0AE2H         LINE#         369
  C:0AE2H         LINE#         370
  C:0AE7H         LINE#         371
  C:0AEDH         LINE#         372
  C:0AEEH         LINE#         374
  C:0AEEH         LINE#         375
  C:0AF4H         LINE#         376
  C:0AFAH         LINE#         377
  C:0AFBH         LINE#         379
  C:0AFBH         LINE#         380
  C:0B01H         LINE#         381
  C:0B07H         LINE#         382
  C:0B07H         LINE#         384
  C:0B07H         LINE#         386
  -------         ENDPROC       _DIG1
  -------         PROC          _DIG2
  D:0050H         SYMBOL        num
  C:0B08H         LINE#         387
  C:0B0CH         LINE#         388
BL51 BANKED LINKER/LOCATER V6.22.2.0                                                  10/25/2022  13:54:05  PAGE 8


  C:0B0CH         LINE#         389
  C:0B40H         LINE#         390
  C:0B40H         LINE#         392
  C:0B40H         LINE#         393
  C:0B46H         LINE#         394
  C:0B4CH         LINE#         395
  C:0B4DH         LINE#         397
  C:0B4DH         LINE#         398
  C:0B52H         LINE#         399
  C:0B58H         LINE#         400
  C:0B59H         LINE#         402
  C:0B59H         LINE#         403
  C:0B5FH         LINE#         404
  C:0B65H         LINE#         405
  C:0B66H         LINE#         407
  C:0B66H         LINE#         408
  C:0B6CH         LINE#         409
  C:0B72H         LINE#         410
  C:0B73H         LINE#         412
  C:0B73H         LINE#         413
  C:0B79H         LINE#         414
  C:0B7FH         LINE#         415
  C:0B80H         LINE#         417
  C:0B80H         LINE#         418
  C:0B86H         LINE#         419
  C:0B8CH         LINE#         420
  C:0B8DH         LINE#         422
  C:0B8DH         LINE#         423
  C:0B93H         LINE#         424
  C:0B99H         LINE#         425
  C:0B9AH         LINE#         427
  C:0B9AH         LINE#         428
  C:0B9FH         LINE#         429
  C:0BA5H         LINE#         430
  C:0BA6H         LINE#         432
  C:0BA6H         LINE#         433
  C:0BACH         LINE#         434
  C:0BB2H         LINE#         435
  C:0BB3H         LINE#         437
  C:0BB3H         LINE#         438
  C:0BB9H         LINE#         439
  C:0BBFH         LINE#         440
  C:0BBFH         LINE#         442
  C:0BBFH         LINE#         444
  -------         ENDPROC       _DIG2
  -------         PROC          _DIG3
  D:0052H         SYMBOL        num
  C:0BC0H         LINE#         445
  C:0BC4H         LINE#         446
  C:0BC4H         LINE#         447
  C:0BF8H         LINE#         448
  C:0BF8H         LINE#         450
  C:0BF8H         LINE#         451
  C:0BFEH         LINE#         452
  C:0C04H         LINE#         453
  C:0C05H         LINE#         455
  C:0C05H         LINE#         456
BL51 BANKED LINKER/LOCATER V6.22.2.0                                                  10/25/2022  13:54:05  PAGE 9


  C:0C0AH         LINE#         457
  C:0C10H         LINE#         458
  C:0C11H         LINE#         460
  C:0C11H         LINE#         461
  C:0C17H         LINE#         462
  C:0C1DH         LINE#         463
  C:0C1EH         LINE#         465
  C:0C1EH         LINE#         466
  C:0C24H         LINE#         467
  C:0C2AH         LINE#         468
  C:0C2BH         LINE#         470
  C:0C2BH         LINE#         471
  C:0C31H         LINE#         472
  C:0C37H         LINE#         473
  C:0C38H         LINE#         475
  C:0C38H         LINE#         476
  C:0C3EH         LINE#         477
  C:0C44H         LINE#         478
  C:0C45H         LINE#         480
  C:0C45H         LINE#         481
  C:0C4BH         LINE#         482
  C:0C51H         LINE#         483
  C:0C52H         LINE#         485
  C:0C52H         LINE#         486
  C:0C57H         LINE#         487
  C:0C5DH         LINE#         488
  C:0C5EH         LINE#         490
  C:0C5EH         LINE#         491
  C:0C64H         LINE#         492
  C:0C6AH         LINE#         493
  C:0C6BH         LINE#         495
  C:0C6BH         LINE#         496
  C:0C71H         LINE#         497
  C:0C77H         LINE#         498
  C:0C77H         LINE#         500
  C:0C77H         LINE#         501
  -------         ENDPROC       _DIG3
  -------         PROC          _DIG4
  D:0054H         SYMBOL        num
  C:0C78H         LINE#         502
  C:0C7CH         LINE#         503
  C:0C7CH         LINE#         504
  C:0CB0H         LINE#         505
  C:0CB0H         LINE#         507
  C:0CB0H         LINE#         508
  C:0CB6H         LINE#         509
  C:0CBCH         LINE#         510
  C:0CBDH         LINE#         512
  C:0CBDH         LINE#         513
  C:0CC2H         LINE#         514
  C:0CC8H         LINE#         515
  C:0CC9H         LINE#         517
  C:0CC9H         LINE#         518
  C:0CCFH         LINE#         519
  C:0CD5H         LINE#         520
  C:0CD6H         LINE#         522
  C:0CD6H         LINE#         523
BL51 BANKED LINKER/LOCATER V6.22.2.0                                                  10/25/2022  13:54:05  PAGE 10


  C:0CDCH         LINE#         524
  C:0CE2H         LINE#         525
  C:0CE3H         LINE#         527
  C:0CE3H         LINE#         528
  C:0CE9H         LINE#         529
  C:0CEFH         LINE#         530
  C:0CF0H         LINE#         532
  C:0CF0H         LINE#         533
  C:0CF6H         LINE#         534
  C:0CFCH         LINE#         535
  C:0CFDH         LINE#         537
  C:0CFDH         LINE#         538
  C:0D03H         LINE#         539
  C:0D09H         LINE#         540
  C:0D0AH         LINE#         542
  C:0D0AH         LINE#         543
  C:0D0FH         LINE#         544
  C:0D15H         LINE#         545
  C:0D16H         LINE#         547
  C:0D16H         LINE#         548
  C:0D1CH         LINE#         549
  C:0D22H         LINE#         550
  C:0D23H         LINE#         552
  C:0D23H         LINE#         553
  C:0D29H         LINE#         554
  C:0D2FH         LINE#         555
  C:0D2FH         LINE#         557
  C:0D2FH         LINE#         559
  -------         ENDPROC       _DIG4
  -------         PROC          POINT
  C:116CH         LINE#         561
  C:116CH         LINE#         562
  C:116CH         LINE#         563
  C:1177H         LINE#         564
  -------         ENDPROC       POINT
  -------         PROC          TIMERINIT
  C:1178H         LINE#         566
  C:1178H         LINE#         567
  C:1178H         LINE#         568
  C:117BH         LINE#         570
  -------         ENDPROC       TIMERINIT
  -------         PROC          MAIN
  -------         DO            
  D:0056H         SYMBOL        i
  -------         ENDDO         
  C:0697H         LINE#         580
  C:0697H         LINE#         581
  C:0697H         LINE#         582
  C:069DH         LINE#         583
  C:06A0H         LINE#         584
  C:06A3H         LINE#         586
  C:06A6H         LINE#         587
  C:06A9H         LINE#         588
  C:06ACH         LINE#         589
  C:06AFH         LINE#         592
  C:06B5H         LINE#         594
  C:06BCH         LINE#         596
BL51 BANKED LINKER/LOCATER V6.22.2.0                                                  10/25/2022  13:54:05  PAGE 11


  C:06BCH         LINE#         597
  C:06BCH         LINE#         599
  C:06D2H         LINE#         600
  C:06D2H         LINE#         601
  C:06D7H         LINE#         602
  C:06E9H         LINE#         603
  C:06EEH         LINE#         604
  C:06FBH         LINE#         606
  C:0700H         LINE#         607
  C:0712H         LINE#         608
  C:0717H         LINE#         609
  C:0724H         LINE#         611
  C:072BH         LINE#         613
  C:073FH         LINE#         614
  C:073FH         LINE#         616
  C:0742H         LINE#         617
  C:0745H         LINE#         618
  C:0748H         LINE#         619
  C:074BH         LINE#         621
  C:074EH         LINE#         622
  C:0754H         LINE#         623
  C:0754H         LINE#         625
  C:0768H         LINE#         626
  C:0768H         LINE#         627
  C:076BH         LINE#         628
  C:076EH         LINE#         629
  C:0771H         LINE#         631
  C:0774H         LINE#         632
  C:077AH         LINE#         633
  C:077AH         LINE#         634
  C:0785H         LINE#         636
  C:079BH         LINE#         637
  C:079BH         LINE#         639
  C:07A0H         LINE#         640
  C:07B2H         LINE#         641
  C:07B7H         LINE#         642
  C:07C4H         LINE#         644
  C:07C9H         LINE#         645
  C:07DBH         LINE#         646
  C:07E0H         LINE#         647
  C:07EDH         LINE#         649
  C:07F4H         LINE#         651
  C:0808H         LINE#         652
  C:0808H         LINE#         653
  C:080BH         LINE#         654
  C:080EH         LINE#         655
  C:0811H         LINE#         656
  C:0814H         LINE#         658
  C:0817H         LINE#         659
  C:081DH         LINE#         660
  C:081DH         LINE#         662
  C:0831H         LINE#         663
  C:0831H         LINE#         664
  C:0834H         LINE#         665
  C:0837H         LINE#         666
  C:083AH         LINE#         668
  C:083DH         LINE#         669
BL51 BANKED LINKER/LOCATER V6.22.2.0                                                  10/25/2022  13:54:05  PAGE 12


  C:0843H         LINE#         670
  C:0843H         LINE#         672
  C:084EH         LINE#         674
  -------         ENDPROC       MAIN
  -------         PROC          RTD_MEASURE_SHOW
  C:0852H         LINE#         678
  C:0852H         LINE#         679
  C:0852H         LINE#         680
  C:085AH         LINE#         682
  C:085DH         LINE#         684
  C:08B6H         LINE#         686
  C:08BEH         LINE#         687
  C:08BEH         LINE#         688
  C:08C4H         LINE#         689
  C:08CAH         LINE#         690
  C:08CAH         LINE#         692
  C:08D2H         LINE#         693
  C:08D2H         LINE#         694
  C:08D8H         LINE#         695
  C:0920H         LINE#         696
  C:0920H         LINE#         698
  C:092BH         LINE#         699
  C:092BH         LINE#         700
  C:0973H         LINE#         701
  C:0979H         LINE#         702
  C:0979H         LINE#         704
  -------         ENDPROC       RTD_MEASURE_SHOW
  -------         PROC          RTD_SHOW
  C:097AH         LINE#         706
  C:097AH         LINE#         707
  C:097AH         LINE#         708
  C:09CAH         LINE#         709
  C:09E4H         LINE#         713
  C:09FDH         LINE#         714
  C:0A21H         LINE#         715
  C:0A24H         LINE#         716
  C:0A48H         LINE#         717
  C:0A4FH         LINE#         719
  -------         ENDPROC       RTD_SHOW
  -------         PROC          TMR0INIT
  C:1043H         LINE#         721
  C:1043H         LINE#         722
  C:1043H         LINE#         724
  C:1049H         LINE#         725
  C:104FH         LINE#         728
  C:1054H         LINE#         729
  C:105AH         LINE#         730
  C:105FH         LINE#         731
  C:1065H         LINE#         734
  C:106BH         LINE#         735
  C:1071H         LINE#         736
  C:1077H         LINE#         737
  C:107DH         LINE#         742
  C:1088H         LINE#         744
  -------         ENDPROC       TMR0INIT
  -------         PROC          TMR1INIT
  C:1089H         LINE#         746
BL51 BANKED LINKER/LOCATER V6.22.2.0                                                  10/25/2022  13:54:05  PAGE 13


  C:1089H         LINE#         747
  C:1089H         LINE#         749
  C:108FH         LINE#         750
  C:1095H         LINE#         753
  C:109AH         LINE#         754
  C:10A0H         LINE#         755
  C:10A5H         LINE#         756
  C:10ABH         LINE#         759
  C:10B1H         LINE#         760
  C:10B7H         LINE#         761
  C:10BDH         LINE#         762
  C:10C3H         LINE#         767
  C:10CEH         LINE#         768
  -------         ENDPROC       TMR1INIT
  -------         ENDMOD        MAIN

  -------         MODULE        ?C?FPADD
  C:0035H         PUBLIC        ?C?FPADD
  C:0031H         PUBLIC        ?C?FPSUB
  -------         ENDMOD        ?C?FPADD

  -------         MODULE        ?C?FPMUL
  C:0126H         PUBLIC        ?C?FPMUL
  -------         ENDMOD        ?C?FPMUL

  -------         MODULE        ?C?FPDIV
  C:022FH         PUBLIC        ?C?FPDIV
  -------         ENDMOD        ?C?FPDIV

  -------         MODULE        ?C?FCAST
  C:02D6H         PUBLIC        ?C?FCASTC
  C:02D1H         PUBLIC        ?C?FCASTI
  C:02CCH         PUBLIC        ?C?FCASTL
  -------         ENDMOD        ?C?FCAST

  -------         MODULE        ?C?CASTF
  C:030AH         PUBLIC        ?C?CASTF
  -------         ENDMOD        ?C?CASTF

  -------         MODULE        ?C?UIDIV
  C:038BH         PUBLIC        ?C?UIDIV
  -------         ENDMOD        ?C?UIDIV

  -------         MODULE        ?C?LMUL
  C:03E0H         PUBLIC        ?C?LMUL
  -------         ENDMOD        ?C?LMUL

  -------         MODULE        ?C?LNEG
  C:042FH         PUBLIC        ?C?LNEG
  -------         ENDMOD        ?C?LNEG

  -------         MODULE        ?C?ULCMP
  C:043DH         PUBLIC        ?C?ULCMP
  -------         ENDMOD        ?C?ULCMP

  -------         MODULE        ?C?ICASE
  C:044EH         PUBLIC        ?C?ICASE
BL51 BANKED LINKER/LOCATER V6.22.2.0                                                  10/25/2022  13:54:05  PAGE 14


  -------         ENDMOD        ?C?ICASE

  -------         MODULE        ?C_IBP
  D:005AH         PUBLIC        ?C_IBP
  -------         ENDMOD        ?C_IBP



FUNCTION REGISTER MASKS


FUNCTION . . . . . . REG MASK
-----------------------------

ANACCONFIG . . . . . @0xe301
CLKCONFIG. . . . . . @0xe301
IOCONFIG . . . . . . @0xe301
LCMINIT. . . . . . . @0xf303
POINT. . . . . . . . @0xe301
SDMCONFIG. . . . . . @0xe301
SDM_LIGHT_CONFIG . . @0xe301
SYSTEMINIT . . . . . @0x8000
TMR0INIT . . . . . . @0xe301
TMR1INIT . . . . . . @0xe301
_DELAY . . . . . . . @0xf000
_DIG1. . . . . . . . @0xf780
_DIG2. . . . . . . . @0xf780
_DIG3. . . . . . . . @0xf780
_DIG4. . . . . . . . @0xf780

*** WARNING L16: UNCALLED SEGMENT, IGNORED FOR OVERLAY PROCESS
    SEGMENT: ?PR?SYSTEMINIT?SYSTEM_FE81001

*** WARNING L16: UNCALLED SEGMENT, IGNORED FOR OVERLAY PROCESS
    SEGMENT: ?PR?TMR1INIT?MAIN

Program Size: data=92.0 xdata=4 code=4477
LINK/LOCATE RUN COMPLETE.  2 WARNING(S),  0 ERROR(S)
